:100000000C9483000C94B8260C94E3260C940E27D1
:100010000C94AF000C94AF000C94AF000C94AF00A4
:100020000C94AF000C94AF000C94AF000C94AF0094
:100030000C94AF000C94AF000C94AF000C94AF0084
:100040000C94AF000C94AF000C945F280C94AF009C
:100050000C94C62B0C94FC2B0C94AF000C94AF00AA
:100060000C94AF000C94AF000C94AF000C94AF0054
:100070000C94AF000C94AF000C94AF000C94FC24D3
:100080000C94AF000C94AF000C94AF000000000182
:100090000200090A00000000040308070000000035
:1000A0000000000000000000000000000102040841
:1000B0001020408001020408102040800102040842
:1000C0001020408001020408102040800202020239
:1000D00002020202040404040404040403030303EC
:1000E00003030303010101010101010100002200DA
:1000F000250028002B0000002100240027002A00F2
:10010000FB056B1D302C2092863A11241FBECFEFC9
:10011000D0E4DEBFCDBF11E0A0E0B1E0E0E7F0E663
:1001200000E00BBF02C007900D92AC38B107D9F7C1
:100130002AE3ACE8B1E001C01D92A638B207E1F7AE
:1001400010E0C3E8D0E004C02197FE010E94712EA8
:10015000C038D107C9F70E94B32C0C9436300C94E8
:100160000000CF93DF931F92CDB7DEB76983DC0128
:10017000ED91FC910280F381E02D41E050E0BE0161
:100180006F5F7F4F09950F90DF91CF91089508958C
:10019000FC011382128288EE93E0A0E0B0E0848339
:1001A0009583A683B7838BE291E09183808380E57A
:1001B000848781E085878AE090E09787868789E059
:1001C00090E0918B808B82E090E0938B828B148AFD
:1001D000158A168A178A118E108E138E128E158E1E
:1001E000148E40E050E0BA01CF010C948A2CFC013F
:1001F00077876687518B408B338B228B08950F93C3
:100200001F93CF93DF93EC01062F142F60E08E85B0
:100210000E94652A3C852D858091DA39882381F0FA
:100220009FB7F8948091DA39813081F58DB380934E
:10023000D8394DB38091D939809584238DBB9FBF28
:100240003CBD2DBD0EBD00000DB407FEFDCF8EB52B
:100250001EBD00000DB407FEFDCF1EB58091DA393A
:10026000882351F09FB7F8942091DA398091D839DA
:10027000213079F48DBB9FBF61E08E850E94652A95
:10028000812FDF91CF911F910F9108959093D839CD
:10029000D7CF8FBFF1CF6F7740E00C94FF0068E1BC
:1002A0000C944B0169E10C944B0169E10E944B01F4
:1002B000682F880F770B880B990B0E94FF2C20E08A
:1002C00030E040E85EE30E94AF2D08958F929F9248
:1002D000AF92BF92EF92FF920F931F93CF93DF9352
:1002E0008C016AE10E944B01C82FD0E0C8010E9436
:1002F00055010E94C72C4B017B01F8016489758967
:10030000868997890E94FF2C24ED30E843E45EE45F
:100310000E94C22CBE0187FD12C06D597109F7FE03
:1003200011C0680D791DCB01DF91CF911F910F9105
:10033000FF90EF90BF90AF909F908F900895645A78
:100340007109EDCF072E000C880B990B0E94FF2C32
:1003500020EB32E748E85FE30E94AF2D0E94C72CF4
:10036000E2CFCF93DF93EC0163E10E944B0190E079
:10037000288D398D821B930BDF91CF910895CF93F8
:10038000DF93EC01E881F9810480F581E02D099586
:10039000892B69F0888D998D0196998F888F60E0FF
:1003A000CE010E944B0190E0DF91CF9108958FEF35
:1003B0009FEFFACF0F931F93CF93DF938C0166E0EB
:1003C0000E944B01D82F67E0C8010E944B01C82F43
:1003D00068E0C8010E944B014C2F50E070E060E0E3
:1003E000762F652F542F44276D2B8A019B01082BF4
:1003F000C901B80120E038E448EE51E00E948C2E9B
:1004000003E10E94312FB901CA01DF91CF911F9101
:100410000F9108956DE10E944B01E82FF0E084E018
:10042000F595E7958A95E1F7EA30F10508F036C0D1
:10043000E45EFD4F0C94712E4F02260254022B02F3
:10044000300235023A023F024402490260EA78E291
:1004500080E090E0089560E471E580E090E0089528
:1004600062E17AE780E090E0089564EE72EA80E06D
:1004700090E0089564E274EF80E090E0089568E40D
:1004800078EE81E090E0089560E970ED83E090E01F
:10049000089560E271EA87E090E00895089568E7C2
:1004A0007EE180E090E0089560EF7CE380E090E002
:1004B00008956CE20C944B01CF93DF93EC0143E879
:1004C00061E80E94FF0062E1CE010E944B0183FDC2
:1004D00003C00E945E28F7CF48E062E9CE010E9487
:1004E000FF0081E090E0DF91CF910895AF92BF923D
:1004F000CF92DF92FF920F931F93CF93DF936C0104
:100500005B01EA0162E20E944B01F82E90E09C013F
:100510002C0F3D1F2F3F310529F020F0CFEFD0E009
:10052000C81BD90B8501AC0EBD1E0A151B0541F079
:10053000F80141918F0160E8C6010E94FF00F5CFEC
:100540004C2F4F0D62EAC6010E94FF00CE01DF91E1
:10055000CF911F910F91FF90DF90CF90BF90AF9000
:1005600008950F931F93CF93DF93EC01E881F981F6
:100570000480F581E02D0995892BB1F06DE0CE0165
:100580000E944B01082F60E0CE010E944B01182F02
:10059000402F6DE8CE010E94FF00812F90E0DF9197
:1005A000CF911F910F9108958FEF9FEFF8CFCF93C9
:1005B000DF93EC017D8F6C8F8A899B89672BA1F17A
:1005C00060E00E94292A40E060ECCE010E94FF001A
:1005D0008A899B8982309105D9F08A309105D1F0C2
:1005E0000B97D1F481E00E9438268A899B8982305A
:1005F0009105A1F08A30910599F00B9799F481E06B
:1006000043E050E06BED75E0DF91CF910C947326E1
:1006100082E0E9CF80E0E7CF8FEFE5CF82E0F0CF57
:1006200080E0EECF8FEFECCF82309105B9F08A30C9
:100630009105B1F00B97B1F481E00E94A2268A895E
:100640009B898230910581F08A30910579F00B9772
:1006500079F481E0DF91CF910C94572682E0EDCFC1
:1006600080E0EBCF8FEFE9CF82E0F4CF80E0F2CFF4
:100670008FEFF0CF41E861E80C94FF0040E861E8BB
:100680000C94FF000E943E030C942426AF92BF926C
:10069000CF92DF92EF92FF920F931F93CF93DF934E
:1006A000EC01DB01CA018C8B9D8BAE8BBF8B6A0189
:1006B0007B01FF0CCC08DC2C76019A01AB016C2D80
:1006C0007C2D8C2D9C2D03E10E94162FA12CE8E49B
:1006D000BE2EF8EECF2EDD24D394E12CF12C00E0D9
:1006E00010E00E94B92E122FC22ED32E7A01A7013C
:1006F0006627772766E8CE010E94FF0077276F2DD7
:100700005E2D4D2D67E8CE010E94FF00412F68E865
:10071000CE01DF91CF911F910F91FF90EF90DF906D
:10072000CF90BF90AF900C94FF00CF92DF92EF92EA
:10073000FF92CF93DF93EC016A017B0161E08E852C
:100740000E94292A61E08E850E94652A88899989FC
:100750008F3F9807B9F061E00E94292A60E08889FC
:100760000E94652A6AE070E080E090E00E94DA284A
:1007700061E088890E94652A6AE070E080E090E08C
:100780000E94DA280E94EE2562E4CE010E944B010D
:10079000823191F5CE010E943E03B701A601CE0140
:1007A0000E94460340E06EE8CE010E94FF0040E058
:1007B0006FE8CE010E94FF006CE0CE010E944B0169
:1007C000482F43606CE8CE010E94FF0044E066EAD7
:1007D000CE010E94FF0040E869E8CE010E94FF00C0
:1007E000CE010E943A0381E090E0DF91CF91FF902B
:1007F000EF90DF90CF90089590E080E0F6CFCF9219
:10080000DF92EF92FF92CF93DF93EC016EE10E94B3
:100810004B01F82ECE010E940A02F2942FE0F22240
:10082000CC24C394D12C02C0CC0CDD1CFA94E2F78A
:100830000D2C000CEE08FF0828EE33E040E050E0FD
:100840000E94522EC701B6010E94522E213131055D
:10085000410551055CF04CE066EACE01DF91CF9195
:10086000FF90EF90DF90CF900C94FF0044E0F4CF26
:100870000F931F93CF93DF938C01EB0166307105CB
:1008800034F06D30710534F56630710529F545ECAD
:1008900061EBC8010E94FF004CE067EBC8010E94B9
:1008A000FF00C6E0D0E06EE1C8010E944B018F70EE
:1008B00094E0CC0FDD1F9A95E1F74C2F482B6EE9A1
:1008C000C8010E94FF00C801DF91CF911F910F91D5
:1008D0000C94FF03CCE0D0E043EC61EBC8010E9434
:1008E000FF004AE067EBC8010E94FF00DCCFCF9217
:1008F000DF92EF92FF920F931F93CF93DF938C01C0
:10090000CB01BA010E94FF2C6B017C0120E030EC8E
:1009100043EF55E40E94C22CD0E0C0E018160CF062
:1009200065C020E030E842E256E4C701B6010E940B
:10093000C22CC1E0D0E018160CF058C020E030EC1A
:1009400043E756E4C701B6010E94C22CC2E0D0E0E2
:1009500018160CF04BC020E030E842EA56E4C7011C
:10096000B6010E94C22CC3E0D0E018160CF03EC0C5
:1009700020E034E244EF56E4C701B6010E94C22CE5
:10098000C4E0D0E0181694F520E034EE42E257E4DB
:10099000C701B6010E94C22CC5E0D0E0181634F59C
:1009A00020E034E244E757E4C701B6010E94C22CBC
:1009B000C6E0D0E01816D4F420E034E244EF57E467
:1009C000C701B6010E94C22CC7E0D0E0181674F42B
:1009D00020E034E244E758E4C701B6010E94C22C8B
:1009E000C9E0D0E0181614F0C8E0D0E06DE1C8010D
:1009F0000E944B018F7094E0CC0FDD1F9A95E1F7B8
:100A00004C2F482B6DE9C8010E94FF00C801DF91FF
:100A1000CF911F910F91FF90EF90DF90CF900C94AA
:100A2000FF030F931F93CF93DF938C01EB0169308A
:100A3000710514F0C8E0D0E06DE1C8010E944B01DF
:100A4000C530D10514F4C5E0D0E02497CC0FDD1FEC
:100A5000482F417F4C2B6DE9C801DF91CF911F9149
:100A60000F910C94FF00CF93DF93EC016EE10E9495
:100A70004B01482F44606EE9CE01DF91CF910C9479
:100A8000FF00CF93DF93EC011B8E1A8E6DE10E9465
:100A90004B01482F4E7F6DE9CE01DF91CF910C9431
:100AA000FF00CF93DF93EC0181E090E09B8F8A8F72
:100AB0006DE1CE010E944B01482F41606DE9CE01EE
:100AC000DF91CF910C94FF000F931F93CF93DF938F
:100AD000EC018B010E943A03CE01012B99F00E9498
:100AE000510540E06DE8CE010E94FF0040E062EA5F
:100AF000CE010E94FF0081E090E0DF91CF911F9135
:100B00000F9108950E944105ECCF0F931F93CF934F
:100B1000DF93EC018B011616170684F40E94510531
:100B2000402F62EACE010E94FF0045E861E8CE0155
:100B3000DF91CF911F910F910C94FF000E9441050E
:100B4000F4CF0F931F93CF93DF93EC0162E10E94E8
:100B50004B01182F482F62E9CE010E94FF0015FDBE
:100B600025C0198E188E8A8D9B8D62E2892B09F41F
:100B700063E1CE010E944B01082F10E060E1CE013D
:100B80000E944B01482F6DE8CE010E94FF00EC8DC2
:100B9000FD8D309711F0C801099540E06DE8CE0158
:100BA000DF91CF911F910F910C94FF00DF91CF91B6
:100BB0001F910F9108958CE891E00C94A105452BAD
:100BC00061F4AB016F30710514F04EE050E057FD59
:100BD00040E0406769E80C94FF00AB0162317105A9
:100BE00014F041E150E04230510514F442E050E08D
:100BF00042504068EFCF8CE891E00C94C8002F92EF
:100C00003F924F925F926F927F928F929F92AF929C
:100C1000BF92CF92DF92EF92FF920F931F93CF93E9
:100C2000DF93CDB7DEB7C857D1090FB6F894DEBF52
:100C30000FBECDBFE9969FAF8EAFE9971A01DC01D9
:100C400018960D911D912D913C911B9761960CAFBB
:100C50001DAF2EAF3FAF61971C960D911D912D9149
:100C60003C911F9709831A832B833C8350960D91E7
:100C70001D912D913C9153970D831E832F833887AF
:100C800054960D911D912D913C91579709871A8784
:100C90002B873C87E6966FAFE697E7967FAFE7979F
:100CA000A85ABF4F6396BFAFAEAF6397FC01E45A3B
:100CB000FF4F6596FFAFEEAF65978C01005A1F4F4F
:100CC00067961FAF0EAF67979C012C593F4F6996EF
:100CD0003FAF2EAF699788599F4F6B969FAF8EAFEE
:100CE0006B97E996AEADBFADE997A459BF4F6D962E
:100CF000BFAFAEAF6D97E996EEADFFADE997E059A6
:100D0000FF4F6F96FFAFEEAF6F97E9960EAD1FAD39
:100D1000E9970C581F4FA1961FAF0EAFA197E99608
:100D20002EAD3FADE99728583F4FA3963FAF2EAF6A
:100D3000A397E9968EAD9FADE99784589F4FA596EE
:100D40009FAF8EAFA597E996AEADBFADE997A0581E
:100D5000BF4FA796BFAFAEAFA797E996EEADFFAD79
:100D6000E997EC57FF4FA996FFAFEEAFA997E99629
:100D70000EAD1FADE99708571F4FAB961FAF0EAFD3
:100D8000AB97E9962EAD3FADE99724573F4FAD960F
:100D90003FAF2EAFAD97E9968EAD9FADE9978057E7
:100DA0009F4FAF969FAF8EAFAF97E996AEADBFADF9
:100DB000E997AC56BF4FE196BFAFAEAFE197E7966C
:100DC000AEADBFADE7970D911D912D913C910D8773
:100DD0001E872F87388B6396EEADFFAD6397008338
:100DE00011832283338361968CAD9DADAEADBFADD3
:100DF000619788589B45A549B842800F911FA21F53
:100E0000B31F4D815E816F81788509851A852B8599
:100E10003C85402751276227732709811A812B813E
:100E20003C81402351236223732309851A852B8536
:100E30003C854027512762277327840F951FA61FE3
:100E4000B71F8C019D0147E0000F111F221F331FA8
:100E50004A95D1F7AC01BD01E9E1769567955795C3
:100E60004795EA95D1F7402B512B622B732B898143
:100E70009A81AB81BC81480F591F6A1F7B1FE7967F
:100E8000AEADBFADE79714960D911D912D913C919C
:100E90001797098B1A8B2B8B3C8B6596EEADFFADAC
:100EA0006597008311832283338389859A85AB8577
:100EB000BC858A5A9844A843B741800F911FA21F4E
:100EC000B31FC980DA80EB80FC800D811E812F81E9
:100ED0003885C026D126E226F326C422D522E62272
:100EE000F722C026D126E226F3268C0D9D1DAE1DCD
:100EF000BF1D8C019D01FCE0000F111F221F331F3D
:100F0000FA95D1F76C017D01A4E1F694E794D794AA
:100F1000C794AA95D1F7C02AD12AE22AF32AC40E8F
:100F2000D51EE61EF71EE796AEADBFADE797189645
:100F30008D919D910D90BC91A02D8D8B9E8BAF8B33
:100F4000B88F6796EEADFFAD679780839183A283DC
:100F5000B3838D819E81AF81B88585529F48AF4D07
:100F6000BB4D0D891E892F89388D800F911FA21FBF
:100F7000B31F49805A806B807C80442655266626A4
:100F800077264C205D206E207F2009811A812B81DD
:100F90003C814026512662267326840D951DA61D90
:100FA000B71D8C019D01EFE03695279517950795A4
:100FB000EA95D1F72C013D01F1E1440C551C661C6A
:100FC000771CFA95D1F7402A512A622A732A4C0CD1
:100FD0005D1C6E1C7F1CE796AEADBFADE7971C96FF
:100FE0008D919D910D90BC91A02D898F9A8FAB8F83
:100FF000BC8F6996EEADFFAD699780839183A28324
:10100000B38389819A81AB81BC8182519143A2448F
:10101000BE43098D1A8D2B8D3C8D800F911FA21F11
:10102000B31F8A019B010C251D252E253F25042178
:101030001521262137210427152726273727800F3A
:10104000911FA21FB31F4C015D011AE0B694A79433
:10105000979487941A95D1F78C019D0186E1000F32
:10106000111F221F331F8A95D1F7082919292A2910
:101070003B29040D151D261D371DE796AEADBFADEE
:10108000E79750968D919D910D90BC91A02D8D8FDD
:101090009E8FAF8FB8A36B96EEADFFAD6B9780833D
:1010A0009183A283B3838155904FA348BA40840FA4
:1010B000951FA61FB71FB701A60144255525662514
:1010C000772540235123622373234C255D256E250C
:1010D0007F25840F951FA61FB71F4C015D0147E0B8
:1010E000880C991CAA1CBB1C4A95D1F7AC01BD0108
:1010F000E9E17695679557954795EA95D1F748299F
:1011000059296A297B29400F511F621F731FE796D7
:10111000AEADBFADE79754968D919D910D90BC916A
:10112000A02D89A39AA3ABA3BCA36D96EEADFFAD92
:101130006D9780839183A283B383865D9943A8478B
:10114000B84B8C0D9D1DAE1DBF1D73016201C026E5
:10115000D126E226F326C422D522E622F722C42491
:10116000D524E624F7248C0D9D1DAE1DBF1D4C011A
:101170005D01FCE0880C991CAA1CBB1CFA95D1F7F8
:101180006C017D01A4E1F694E794D794C794AA95E5
:10119000D1F7C828D928EA28FB28C40ED51EE61E98
:1011A000F71EE796AEADBFADE79758968D919D912E
:1011B0000D90BC91A02D8DA39EA3AFA3B8A76F9651
:1011C000EEADFFAD6F9780839183A283B3838D5E75
:1011D000994BAF4CB745840D951DA61DB71D280131
:1011E000390144265526662677264C205D206E2040
:1011F0007F204026512662267326840D951DA61D4C
:10120000B71D4C015D01EFE0B694A79497948794C5
:10121000EA95D1F72C013D01F1E1440C551C661C07
:10122000771CFA95D1F7482859286A287B284C0C56
:101230005D1C6E1C7F1CE796AEADBFADE7975C965C
:101240008D919D910D90BC91A02D89A79AA7ABA7D8
:10125000BCA7A196EEADFFADA19780839183A28339
:10126000B3838F5F9A46A94BB240800F911FA21F94
:10127000B31F8A019B010C251D252E253F25042126
:101280001521262137210427152726273727800FE8
:10129000911FA21FB31F4C015D011AE0B694A794E1
:1012A000979487941A95D1F78C019D0186E1000FE0
:1012B000111F221F331F8A95D1F7082919292A29BE
:1012C0003B29040D151D261D371DE796AEADBFAD9C
:1012D000E79790968D919D910D90BC91A02D8DA733
:1012E0009EA7AFA7B8ABA396EEADFFADA397808343
:1012F0009183A283B38388529746AF47B649840F40
:10130000951FA61FB71FB701A601442555256625C1
:10131000772540235123622373234C255D256E25B9
:101320007F25840F951FA61FB71F4C015D0147E065
:10133000880C991CAA1CBB1C4A95D1F7AC01BD01B5
:10134000E9E17695679557954795EA95D1F748294C
:1013500059296A297B29400F511F621F731FE79685
:10136000AEADBFADE79794968D919D910D90BC91D8
:10137000A02D89AB9AABABABBCABA596EEADFFADE8
:10138000A59780839183A283B38381559840AB4B0B
:10139000B4478C0D9D1DAE1DBF1D73016201C0269B
:1013A000D126E226F326C422D522E622F722C4243F
:1013B000D524E624F7248C0D9D1DAE1DBF1D4C01C8
:1013C0005D01FCE0880C991CAA1CBB1CFA95D1F7A6
:1013D0006C017D01A4E1F694E794D794C794AA9593
:1013E000D1F7C828D928EA28FB28C40ED51EE61E46
:1013F000F71EE796AEADBFADE79798968D919D919C
:101400000D90BC91A02D8DAB9EABAFABB8AFA796A6
:10141000EEADFFADA79780839183A283B3838F54F2
:10142000944AA109B109840D951DA61DB71D280177
:10143000390144265526662677264C205D206E20ED
:101440007F204026512662267326840D951DA61DF9
:10145000B71D4C015D01EFE0B694A7949794879473
:10146000EA95D1F72C013D01F1E1440C551C661CB5
:10147000771CFA95D1F7482859286A287B284C0C04
:101480005D1C6E1C7F1CE796AEADBFADE7979C96CA
:101490008D919D910D90BC91A02D89AF9AAFABAF6E
:1014A000BCAFA996EEADFFADA99780839183A283CF
:1014B000B38382549842A34AB647800F911FA21F5C
:1014C000B31F8A019B010C251D252E253F250421D4
:1014D0001521262137210427152726273727800F96
:1014E000911FA21FB31F4C015D011AE0B694A7948F
:1014F000979487941A95D1F78C019D0186E1000F8E
:10150000111F221F331F8A95D1F7082919292A296B
:101510003B29040D151D261D371DE796AEADBFAD49
:10152000E797D0968D919D910D90BC91A02D21961D
:101530008CAF9DAFAEAFBFAF2197AB96EEADFFAD19
:10154000AB9780839183A283B3834C015D01FEED51
:101550008F1AFEEE9F0AFFE6AF0AF4E9BF0A840E77
:10156000951EA61EB71EB701A60144255525662562
:10157000772540235123622373234C255D256E2557
:101580007F25480D591D6A1D7B1D4A015B0197E0AF
:10159000880C991CAA1CBB1C9A95D1F7E9E1769599
:1015A000679557954795EA95D1F7482959296A29AA
:1015B0007B29400F511F621F731FE796AEADBFAD71
:1015C000E797D4968D919D910D90BC91A02D259675
:1015D0008CAF9DAFAEAFBFAF2597AD96EEADFFAD73
:1015E000AD9780839183A283B3834C015D01FDE6B7
:1015F0008F1AFEE89F0AF7E6AF0AF2E0BF0A8C0CEA
:101600009D1CAE1CBF1C73016201C026D126E226C0
:10161000F326C422D522E622F722C424D524E624C8
:10162000F724C80CD91CEA1CFB1C46015701FCE03E
:10163000880C991CAA1CBB1CFA95D1F7A4E1F6945E
:10164000E794D794C794AA95D1F7C828D928EA284F
:10165000FB28C40ED51EE61EF71EE796AEADBFAD45
:10166000E797D8968D919D910D90BC91A02D2996CC
:101670008CAF9DAFAEAFBFAF2997AF96EEADFFADCC
:10168000AF9780839183A283B3834C015D01F2E71E
:101690008F1AFCEB9F0AF6E8AF0AF9E5BF0A840C43
:1016A000951CA61CB71C2801390144265526662620
:1016B00077264C205D206E207F2040265126622612
:1016C0007326480C591C6A1C7B1C53014201BFE065
:1016D000B694A79497948794BA95D1F781E1440C76
:1016E000551C661C771C8A95D1F7482859286A280A
:1016F0007B284C0C5D1C6E1C7F1CE796AEADBFAD0D
:10170000E797DC968D919D910D90BC91A02D2D9623
:101710008CAF9DAFAEAFBFAF2D97E196EEADFFADF5
:10172000E19780839183A283B3834C015D01FFED38
:101730008F1AF7EF9F0AFBE4AF0AF6EBBF0A800EA1
:10174000911EA21EB31E8A019B010C251D252E256C
:101750003F25042115212621372104271527262777
:101760003727080D191D2A1D3B1D480159019AE014
:10177000B694A794979487949A95D1F7E6E1000FD1
:10178000111F221F331FEA95D1F7082919292A2989
:101790003B29040D151D261D371D89889A88AB88A5
:1017A000BC888EE9881A8AED980A81EEA80A89E039
:1017B000B80A840E951EA61EB71EB301A2014027CB
:1017C0005127622773274C215D216E217F214425FB
:1017D000552566257725480D591D6A1D7B1D4A0133
:1017E0005B01F5E0880C991CAA1CBB1CFA95D1F78B
:1017F000ABE17695679557954795AA95D1F7482916
:1018000059296A297B29400F511F621F731F8DA020
:101810009EA0AFA0B8A490EC891A9CE4990A9FEB13
:10182000A90A9FE3B90A8C0C9D1CAE1CBF1C680161
:101830007901C426D526E626F726C420D520E62041
:10184000F720C026D126E226F326C80CD91CEA1CB4
:10185000FB1C46015701B9E0880C991CAA1CBB1C53
:10186000BA95D1F787E1F694E794D794C7948A950F
:10187000D1F7C828D928EA28FB28C40ED51EE61EB1
:10188000F71E89AC9AACABACBCACAFEA8A1AA5EA3D
:101890009A0AA1EAAA0AA9EDBA0A840C951CA61C08
:1018A000B71C2A013B014C245D246E247F24402276
:1018B0005122622273224426552666267726480C3A
:1018C000591C6A1C7B1C530142019EE0880C991C28
:1018D000AA1CBB1C9A95D1F7E2E1769467945794C1
:1018E0004794EA95D1F7482859286A287B284C0C58
:1018F0005D1C6E1C7F1C8D849E84AF84B888B6E509
:101900008B1AB8E39B0AB9E4AB0AB6E1BB0A800EB6
:10191000911EA21EB31E97018601042515252625BA
:10192000372504231523262337230C251D252E2593
:101930003F25080D191D2A1D3B1D48015901FCE0DA
:10194000B694A79497948794FA95D1F7A4E1000FE1
:10195000111F221F331FAA95D1F7082919292A29F7
:101960003B29040D151D261D371D89A09AA0ABA08B
:10197000BCA0E3EA8E1AEFEE9E0AE0EDAE0AE9E2C1
:10198000BE0A840E951EA61EB71EB301A2014027F3
:101990005127622773274C215D216E217F21442529
:1019A000552566257725480D591D6A1D7B1D4A0161
:1019B0005B01B5E0880C991CAA1CBB1CBA95D1F739
:1019C0008BE176956795579547958A95D1F7482984
:1019D00059296A297B29400F511F621F731F8DA847
:1019E0009EA8AFA8B8ACFDEA8F1AFBEE9F0AFBEBEE
:1019F000AF0AFDEFBF0A8C0C9D1CAE1CBF1C68011A
:101A00007901C426D526E626F726C420D520E6206F
:101A1000F720C026D126E226F326C80CD91CEA1CE2
:101A2000FB1C4601570199E0880C991CAA1CBB1CA1
:101A30009A95D1F7E7E1F694E794D794C794EA959D
:101A4000D1F7C828D928EA28FB28C40ED51EE61EDF
:101A5000F71E2D968CAC9DACAEACBFAC2D978FE72E
:101A6000881A89E1980A8EE5A80A87E2B80A840CE8
:101A7000951CA61CB71C2A013B014C245D246E2436
:101A80007F24402251226222732244265526662654
:101A90007726480C591C6A1C7B1C53014201FEE04E
:101AA000880C991CAA1CBB1CFA95D1F7A2E176946C
:101AB000679457944794AA95D1F7482859286A28DB
:101AC0007B284C0C5D1C6E1C7F1C8D8C9E8CAF8CFF
:101AD000B8A098E3891A94E0990A9CE2A90A98E1CF
:101AE000B90A800E911EA21EB31E9701860104251D
:101AF00015252625372504231523262337230C25D2
:101B00001D252E253F25080D191D2A1D3B1D4801A9
:101B10005901BCE0B694A79497948794BA95D1F7ED
:101B200084E1000F111F221F331F8A95D1F7082966
:101B300019292A293B29040D151D261D371D89A8A1
:101B40009AA8ABA8BCA8AAE18A1AA2E39A0AAEE1B5
:101B5000AA0AAEEDBA0A840E951EA61EB71EB301E0
:101B6000A20140275127622773274C215D216E2156
:101B70007F214425552566257725480D591D6A1D69
:101B80007B1D4A015B0195E0880C991CAA1CBB1CBB
:101B90009A95D1F7EBE17695679557954795EA9534
:101BA000D1F7482959296A297B29400F511F621F03
:101BB000731F29968CAC9DACAEACBFAC2997BAE232
:101BC0008B1AB8EF9B0AB8ECAB0ABCE3BB0A8C0CCF
:101BD0009D1CAE1CBF1C68017901C426D526E626D3
:101BE000F726C420D520E620F720C026D126E226FD
:101BF000F326C80CD91CEA1CFB1C46015701F9E06E
:101C0000880C991CAA1CBB1CFA95D1F7A7E1F69485
:101C1000E794D794C794AA95D1F7C828D928EA2879
:101C2000FB28C40ED51EE61EF71E898C9A8CAB8C41
:101C3000BC8CE9E78E1AE2EF9E0AEAE2AE0AEBE01C
:101C4000BE0A840C951CA61CB71C2A013B014C241F
:101C50005D246E247F244022512262227322442676
:101C6000552666267726480C591C6A1C7B1C530196
:101C70004201BEE0880C991CAA1CBB1CBA95D1F786
:101C800082E176946794579447948A95D1F74828CF
:101C900059286A287B284C0C5D1C6E1C7F1C8DA467
:101CA0009EA4AFA4B8A8F3E18F1AFBEE9F0AF5EA51
:101CB000AF0AFAEBBF0A800E911EA21EB31E970157
:101CC00086010425152526253725042315232623DB
:101CD00037230C251D252E253F25080D191D2A1DEE
:101CE0003B1D480159019CE0B694A79497948794B2
:101CF0009A95D1F7E4E1000F111F221F331FEA95D7
:101D0000D1F7082919292A293B29040D151D261D5B
:101D1000371D25968CAC9DACAEACBFAC25978BEF38
:101D2000881A86E1980A8CE1A80A86E5B80A840E2A
:101D3000951EA61EB71EB301A20140275127622798
:101D400073274C215D216E217F2144255525662571
:101D50007725480D591D6A1D7B1D4A015B01F5E081
:101D6000880C991CAA1CBB1CFA95D1F7ABE176959F
:101D7000679557954795AA95D1F7482959296A2912
:101D80007B29400F511F621F731F8D889E88AF886B
:101D9000B88C98E0891A9CE5990A90E1A90A93E029
:101DA000B90A8C0C9D1CAE1CBF1C68017901C426AD
:101DB000D526E626F726C420D520E620F720C02623
:101DC000D126E226F326C80CD91CEA1CFB1C4601CE
:101DD0005701B9E0880C991CAA1CBB1CBA95D1F715
:101DE00087E1F694E794D794C7948A95D1F7C828E9
:101DF000D928EA28FB28C40ED51EE61EF71E89A4A2
:101E00009AA4ABA4BCA4A7E28A1AADEF9A0AA0E9EF
:101E1000AA0AA8E9BA0A840C951CA61CB71C2A01B8
:101E20003B014C245D246E247F24402251226222F7
:101E300073224426552666267726480C591C6A1CB0
:101E40007B1C530142019EE0880C991CAA1CBB1C00
:101E50009A95D1F7E2E17694679457944794EA957E
:101E6000D1F7482859286A287B284C0C5D1C6E1C29
:101E70007F1C4601570184249524A624B72421966B
:101E80008CAD9DADAEADBFAD21978657934BA54DA3
:101E9000B247800F911FA21FB31F95018401042335
:101EA0001523262337230C251D252E253F25800F9E
:101EB000911FA21FB31F8C019D01FCE03695279551
:101EC00017950795FA95D1F7E5960CAF1DAF2EAF94
:101ED0003FAFE5978C019D01A4E1000F111F221F68
:101EE000331FAA95D1F7E5968CAD9DADAEADBFADD4
:101EF000E597082B192B2A2B3B2B040D151D261DAE
:101F0000371D89A19AA1ABA1BCA18E5B964CA540BF
:101F1000B109840F951FA61FB71F80269126A22600
:101F2000B326880E991EAA1EBB1ED501C40144E02B
:101F3000880F991FAA1FBB1F4A95D1F75CE1B69481
:101F4000A794979487945A95D1F7882A992AAA2A10
:101F5000BB2A800E911EA21EB31E4DA55EA56FA5C5
:101F600078A94F5759406E4878474C0D5D1D6E1D3E
:101F70007F1D73016201C026D126E226F326C82404
:101F8000D924EA24FB24C40ED51EE61EF71EB70191
:101F9000A601EBE0440F551F661F771FEA95D1F7A6
:101FA000F5E1F694E794D794C794FA95D1F7C42A4B
:101FB000D52AE62AF72AC80CD91CEA1CFB1C49AD15
:101FC0005AAD6BAD7CAD4E5D5E4962467249440EC2
:101FD000551E661E771EB901A801482559256A2598
:101FE0007B254C255D256E257F25440E551E661EDE
:101FF000771ED20123013D014C0C5D1C6E1C7F1C21
:1020000029964CAD5DAD6EAD7FAD2997445F574CC1
:102010006A417240400F511F621F731F9501840176
:102020000C251D252E253F2504251525262537257C
:10203000040F151F261F371FB901A801A9E07695C7
:10204000679557954795AA95D1F7B7E1000F111FEE
:10205000221F331FBA95D1F7042B152B262B372BB4
:10206000040D151D261D371D49895A896B897C89E8
:102070004C5B554161447B45480D591D6A1D7B1DD4
:102080004601570184249524A624B724802691264E
:10209000A226B326840E951EA61EB71EB501A40166
:1020A00084E0440F551F661F771F8A95D1F79CE186
:1020B000B694A794979487949A95D1F7842A952AF1
:1020C000A62AB72A800E911EA21EB31E4D8D5E8DCC
:1020D0006F8D78A1475550436142744BC40ED51E95
:1020E000E61EF71EB301A20140275127622773277E
:1020F000482559256A257B254C0D5D1D6E1D7F1DCC
:10210000DB01CA01EBE0880F991FAA1FBB1FEA95EC
:10211000D1F7F5E17695679557954795FA95D1F7FB
:10212000482B592B6A2B7B2B480D591D6A1D7B1D93
:10213000C9A4DAA4EBA4FCA4B0EACB1AB4EBDB0A82
:10214000B4E4EB0AB9E0FB0A4C0C5D1C6E1C7F1C6E
:1021500068017901C824D924EA24FB24C426D526A1
:10216000E626F7264C0C5D1C6E1C7F1CF201230139
:102170003F01440E551E661E771ECDA8DEA8EFA8AF
:10218000F8ACF0E9CF1AF3E4DF0AF0E4EF0AF1E487
:10219000FF0AC00ED11EE21EF31E95018401042722
:1021A00015272627372704251525262537250C0D25
:1021B0001D1D2E1D3F1D68017901A9E0F694E794CD
:1021C000D794C794AA95D1F7B7E1000F111F221F2A
:1021D000331FBA95D1F70C291D292E293F29040D4B
:1021E000151D261D371D2596CCACDDACEEACFFAC25
:1021F00025978AE3C81A81E8D80A84E6E80A87EDB9
:10220000F80AC80CD91CEA1CFB1C4A015B01842497
:102210009524A624B72480269126A226B3268C0CCA
:102220009D1CAE1CBF1C7501640184E0CC0CDD1C40
:10223000EE1CFF1C8A95D1F79CE1B694A794979465
:1022400087949A95D1F78C289D28AE28BF28800EB8
:10225000911EA21EB31ECD84DE84EF84F88896E022
:10226000C91A98EDD90A9EE5E90A95E1F90AC40E62
:10227000D51EE61EF71EB301A20140275127622793
:102280007327482559256A257B254C0D5D1D6E1D3C
:102290007F1D6A017B01EBE0CC0CDD1CEE1CFF1CFA
:1022A000EA95D1F7F5E17695679557954795FA95B3
:1022B000D1F74C295D296E297F29480D591D6A1DCA
:1022C0007B1DC98CDA8CEB8CFC8CABE7CA1AAFECAB
:1022D000DA0AA0E1EA0AABE2FA0A4C0C5D1C6E1CB9
:1022E0007F1C68017901C824D924EA24FB24C42670
:1022F000D526E626F7264C0C5D1C6E1C7F1CF201D1
:1023000023013F01440E551E661E771ECDA0DEA0A0
:10231000EFA0F8A4FBEFCF1AF2EEDF0AF7E7EF0A1F
:10232000FBEFFF0AC00ED11EE21EF31E95018401D1
:102330000427152726273727042515252625372581
:102340000C0D1D1D2E1D3F1D68017901A9E0F6949D
:10235000E794D794C794AA95D1F7B7E1000F111F5E
:10236000221F331FBA95D1F70C291D292E293F2989
:10237000040D151D261D371DC9A8DAA8EBA8FCA859
:1023800087ECC81A8FE2D80A8BE2E80A86E2F80ADC
:10239000C80CD91CEA1CFB1C4A015B01842495244F
:1023A000A624B72480269126A226B3268C0C9D1C39
:1023B000AE1CBF1C7501640184E0CC0CDD1CEE1C5E
:1023C000FF1C8A95D1F79CE1B694A79497948794C3
:1023D0009A95D1F78C289D28AE28BF28800E911E93
:1023E000A21EB31E2196CCACDDACEEACFFAC2197A7
:1023F0009BE1C91A96E6D90A94E2E90A99E1F90A39
:10240000C40ED51EE61EF71EB301A20140275127B8
:1024100062277327482559256A257B254C0D5D1DAC
:102420006E1D7F1D6A017B01EBE0CC0CDD1CEE1CF8
:10243000FF1CEA95D1F7F5E1769567955795479595
:10244000FA95D1F74C295D296E297F29480D591D30
:102450006A1D7B1D2D96CCACDDACEEACFFAC2D9790
:10246000A8E0CA1AA3E8DA0AADE5EA0AA0EEFA0A79
:102470004C0C5D1C6E1C7F1C68017901C824D9249A
:10248000EA24FB24C426D526E626F7264C0C5D1C40
:102490006E1C7F1CF20123013F01440E551E661E77
:1024A000771ECD88DE88EF88F88CFBE9CF1AF9EA31
:1024B000DF0AF3E5EF0AFBE3FF0AC00ED11EE21EBE
:1024C000F31E9501840104271527262737270425A5
:1024D0001525262537250C0D1D1D2E1D3F1D6801B8
:1024E0007901A9E0F694E794D794C794AA95D1F717
:1024F000B7E1000F111F221F331FBA95D1F70C2926
:102500001D292E293F29040D151D261D371DCD849B
:10251000DE84EF84F8888CEBC81A8DEDD80A86ED3E
:10252000E80A8BE0F80AC80CD91CEA1CFB1C4A011B
:102530005B0180949094A094B094802A912AA22A5E
:10254000B32A84249524A624B7248C0C9D1CAE1C8D
:10255000BF1C7501640186E0CC0CDD1CEE1CFF1C69
:102560008A95D1F79AE1B694A794979487949A950F
:10257000D1F78C289D28AE28BF28800E911EA21E60
:10258000B31EC9A4DAA4EBA4FCA499E6C91AD10825
:1025900095EDE90A9CEBF90AC40ED51EE61EF71E5E
:1025A000B301A2014095509560957095482959292D
:1025B0006A297B2940275127622773274C0D5D1D0F
:1025C0006E1D7F1D6A017B01EAE0CC0CDD1CEE1C58
:1025D000FF1CEA95D1F7F6E17695679557954795F3
:1025E000FA95D1F74C295D296E297F29480D591D8F
:1025F0006A1D7B1D2996CCACDDACEEACFFAC2997F7
:10260000A9E5CA1AACEDDA0AABE6EA0AA4E5FA0AC9
:10261000C40CD51CE61CF71C2801390140945094C9
:1026200060947094442A552A662A772A48245924AB
:102630006A247B244C0C5D1C6E1C7F1C73016201A0
:10264000AFE0CC0CDD1CEE1CFF1CAA95D1F7B1E16C
:102650007694679457944794BA95D1F74C285D289F
:102660006E287F28440E551E661E771EC9A0DAA06C
:10267000EBA0FCA0B7ECCB1ABFE5DB0ABCE6EB0A8B
:10268000B3E0FB0AC00ED11EE21EF31E95018401C9
:10269000009510952095309504291529262937296C
:1026A00004271527262737270C0D1D1D2E1D3F1D1E
:1026B000680179018BE0F694E794D794C7948A95E2
:1026C000D1F795E1000F111F221F331F9A95D1F703
:1026D0000C291D292E293F29040D151D261D371DE6
:1026E0002196CCACDDACEEACFFAC2197EDE3CE1A7D
:1026F000E6EADE0AE4EAEE0AEAE9FE0AC80CD91CB8
:10270000EA1CFB1C4A015B0180949094A094B09455
:10271000802A912AA22AB32A84249524A624B724A5
:102720008C0C9D1CAE1CBF1C75016401E6E0CC0C3A
:10273000DD1CEE1CFF1CEA95D1F7FAE1B694A794D4
:1027400097948794FA95D1F78C289D28AE28BF28B6
:10275000800E911EA21EB31EC98CDA8CEB8CFC8CF1
:10276000FEE6CF1AF3E3DF0AF3EFEF0AF0E7FF0A22
:10277000C40ED51EE61EF71EB301A201409550956A
:1027800060957095482959296A297B294027512746
:10279000622773274C0D5D1D6E1D7F1D6A017B0135
:1027A000AAE0CC0CDD1CEE1CFF1CAA95D1F7B6E10B
:1027B0007695679557954795BA95D1F74C295D2938
:1027C0006E297F29480D591D6A1D7B1DCDA8DEA8E5
:1027D000EFA8F8AC83E8C81A8BE0D80A80E1E80AD1
:1027E000F108C40CD51CE61CF71C280139014094E3
:1027F000509460947094442A552A662A772A482473
:1028000059246A247B244C0C5D1C6E1C7F1C7301B4
:1028100062018FE0CC0CDD1CEE1CFF1C8A95D1F709
:1028200091E176946794579447949A95D1F74C2800
:102830005D286E287F28440E551E661E771EC988A7
:10284000DA88EB88FC889FE2C91A92EAD90A9BE7EA
:10285000E90A9AE7F90AC00ED11EE21EF31E95019D
:102860008401009510952095309504291529262975
:10287000372904271527262737270C0D1D1D2E1D48
:102880003F1D68017901EBE0F694E794D794C79473
:10289000EA95D1F7F5E1000F111F221F331FFA95BA
:1028A000D1F70C291D292E293F29040D151D261DA0
:1028B000371DCDA4DEA4EFA4F8A8A1EBCA1AA1E8A5
:1028C000DA0AA7E5EA0AA0E9FA0AC80CD91CEA1C48
:1028D000FB1C4A015B0180949094A094B094802AE0
:1028E000912AA22AB32A84249524A624B7248C0CE6
:1028F0009D1CAE1CBF1C75016401A6E0CC0CDD1C48
:10290000EE1CFF1CAA95D1F7BAE1B694A794979450
:102910008794BA95D1F78C289D28AE28BF28800EC1
:10292000911EA21EB31E2D968CAD9DADAEADBFAD5A
:102930002D9780529941A34DB140840F951FA61F3A
:10294000B71FB301A2014095509560957095482935
:1029500059296A297B294027512762277327840F29
:10296000951FA61FB71F6C017D014AE0CC0CDD1C32
:10297000EE1CFF1C4A95D1F7AC01BD01E6E176954E
:10298000679557954795EA95D1F74C295D296E29AA
:102990007F29480D591D6A1D7B1D8DA19EA1AFA1E8
:1029A000B8A58C5E9C4BAE4FBC45840D951DA61DF5
:1029B000B71D280139014094509460947094442AC2
:1029C000552A662A772A482459246A247B24840DB0
:1029D000951DA61DB71D6C017D01FFE0CC0CDD1C13
:1029E000EE1CFF1CFA95D1F72C013D01A1E1769474
:1029F000679457944794AA95D1F74C285D286E2880
:102A00007F28440E551E661E771E25968CAD9DAD03
:102A1000AEADBFAD25978F559E4EA74FB14B800FE2
:102A2000911FA21FB31F9501840100951095209559
:102A30003095042915292629372904271527262703
:102A40003727800F911FA21FB31F6C017D011BE070
:102A5000F694E794D794C7941A95D1F78C019D0109
:102A600085E1000F111F221F331F8A95D1F70C2912
:102A70001D292E293F29040D151D261D371D8D8D5D
:102A80009E8DAF8DB8A18E579148AC4AB840880D45
:102A9000991DAA1DBB1D4A015B0180949094A094CE
:102AA000B094802A912AA22AB32A84249524A624A9
:102AB000B724880D991DAA1DBB1D6C017D01E6E0A0
:102AC000CC0CDD1CEE1CFF1CEA95D1F74C015D011E
:102AD000FAE1B694A79497948794FA95D1F78C2845
:102AE0009D28AE28BF28800E911EA21EB31E89AD60
:102AF0009AADABADBCAD8B5C9D40A54CB244840F90
:102B0000951FA61FB71FB301A20140955095609570
:102B10007095482959296A297B294027512762271E
:102B20007327840F951FA61FB71F6C017D014AE014
:102B3000CC0CDD1CEE1CFF1C4A95D1F7AC01BD018D
:102B4000E6E17695679557954795EA95D1F74C2933
:102B50005D296E297F29480D591D6A1D7B1D8D89B0
:102B60009E89AF89B88D85549D42A842B54D840D8C
:102B7000951DA61DB71D28013901409450946094FD
:102B80007094442A552A662A772A482459246A24AC
:102B90007B24840D951DA61DB71D6C017D01FFE0F2
:102BA000CC0CDD1CEE1CFF1CFA95D1F72C013D016D
:102BB000A1E17694679457944794AA95D1F74C284D
:102BC0005D286E287F28440E551E661E771E89A933
:102BD0009AA9ABA9BCA98F569C42A947B441800FC2
:102BE000911FA21FB31F9501840100951095209598
:102BF0003095042915292629372904271527262742
:102C00003727800F911FA21FB31F6C017D011BE0AE
:102C1000F694E794D794C7941A95D1F78C019D0147
:102C200085E1000F111F221F331F8A95D1F70C2950
:102C30001D292E293F29040D151D261D371D6196BE
:102C40008CAD9DADAEADBFAD6197880D991DAA1D30
:102C5000BB1D61968CAF9DAFAEAFBFAF6197898151
:102C60009A81AB81BC81800F911FA21FB31F898302
:102C70009A83AB83BC830D811E812F813885040D1F
:102C8000151D261D371D0D831E832F8338878985CB
:102C90009A85AB85BC85840F951FA61FB71F8987B2
:102CA0009A87AB87BC87E796AEADBFADE797A05CD0
:102CB000BF4FE796BFAFAEAFE797B0E42B1A31082E
:102CC00011F00C94DF0661960CAD1DAD2EAD3FAD3D
:102CD0006197E996AEADBFADE99718960D931D9338
:102CE0002D933C931B9709811A812B813C811C9663
:102CF0000D931D932D933C931F970D811E812F8162
:102D0000388550960D931D932D933C9353970985C9
:102D10001A852B853C8554960D931D932D933C93DA
:102D20005797E7968EAD9FADE797C858DF4F0FB620
:102D3000F894DEBF0FBECDBFDF91CF911F910F91F1
:102D4000FF90EF90DF90CF90BF90AF909F908F90CB
:102D50007F906F905F904F903F902F900895CF930A
:102D6000DF93FC0181E093E2A5E4B7E680879187D9
:102D7000A287B38789E89BEAADECBFEE848795878D
:102D8000A687B7878EEF9CEDAAEBB8E9808B918B75
:102D9000A28BB38B86E794E5A2E3B0E1848B958B9D
:102DA000A68BB78B10821182128213821482158235
:102DB00016821782DF01A85ABF4F80E4ED01982FD9
:102DC00019929A95E9F77896DF011D928A95E9F7AD
:102DD000DF91CF9108958F929F92AF92BF92EF9221
:102DE000FF920F931F93CF93DF93EC017B018A0136
:102DF00088819981AA81BB8170E060E04A015B0112
:102E0000880E991EAA1EBB1E2FE1B22288829982CB
:102E1000AA82BB8288169906AA06BB0668F48C8033
:102E20009D80AE80BF802FEF821A920AA20AB20A5A
:102E30008C829D82AE82BF828F739927AA27BB277F
:102E40000097A105B10579F120E4822E912CA12CE7
:102E5000B12C881A990AAA0ABB0A48968C0F9D1FA2
:102E6000481559056A057B0570F4A801B701DF9183
:102E7000CF911F910F91FF90EF90BF90AF909F90D7
:102E80008F900C940830A401B7010E940830E80C20
:102E9000F91C0819190940E450E0BE01685E7F4F33
:102EA000CE010E94FF050034110548F0A801407CC6
:102EB000B701CE010E94FF057C010F731127A80105
:102EC000B701CE014896D3CFEF92FF920F931F9395
:102ED000CF93DF938C01EB01488159816A817B811B
:102EE0004F73552766277727DB01CA010196A11D7D
:102EF000B11D4C0F5D1F20E8FA01208F40E450E027
:102F000060E070E0481B590B6A0B7B0B7E01F8E117
:102F1000EF0EF11C4830510561057105A0F448968B
:102F200070E060E08C0F9D1F0E94113040E450E083
:102F3000B701CE010E94FF0540E450E060E070E080
:102F400080E090E0DC0148505109489670E060E074
:102F50008C0F9D1F0E94113088819981AA81BB81AD
:102F600023E0880F991FAA1FBB1F2A95D1F78883DA
:102F70009983AA83BB83FE01E05BFF4F8083319678
:102F800090833196A0833196B0833C812D819E81C0
:102F90008F8131963083319620833196908331969C
:102FA000808340E450E0B701CE010E94FF05888590
:102FB000F8018083898581838A8582838B858383D9
:102FC0008C8584838D8585838E8586838F85878395
:102FD00088898087898981878A8982878B89838785
:102FE0008C8984878D8985878E8986878F89878755
:102FF00088E9FE0111928A95E9F7DF91CF911F913F
:103000000F91FF90EF900895CF92DF92EF92FF9291
:103010000F931F93CF93DF93CDB7DEB7C859D10974
:103020000FB6F894DEBF0FBECDBF7C016B0180E10F
:1030300090E00E9439278C01CE0101960E94AF16C4
:10304000A601B701CE0101960E94EB16BE016F5F8B
:103050007F4FC8010E946417C801C856DF4F0FB6E2
:10306000F894DEBF0FBECDBFDF91CF911F910F91BE
:10307000FF90EF90DF90CF9008951F93CF93DF9351
:10308000EC01162F0E941830181739F0612FCE016D
:10309000DF91CF911F910C942030DF91CF911F9140
:1030A00008950C941830DC01ED91FC910190F081B1
:1030B000E02D099461E08CE00C94652A60E08CE0DE
:1030C0000C94652A61E08DE00C94652A60E08DE047
:1030D0000C94652A0F931F93CF93DF938C01EC011F
:1030E000892B11F4C1E0D0E01C161D060CF561E03F
:1030F0008CE00E94652A60E08DE00E94652A64E60B
:1031000070E080E090E00E94DA2860E08CE00E94AD
:10311000652A61E08DE00E94652A64E670E080E047
:1031200090E00E94DA2801151105F1F22197DCCF19
:1031300060E08CE00E94652A60E08DE0DF91CF9135
:103140001F910F910C94652A0E9462180E945E18CC
:103150006AE070E080E090E00E94DA280E945A184D
:103160000E94661865E070E080E090E00E94DA2836
:10317000EBCF0F931F93CF93DF938C01EC01892B3F
:1031800011F4C1E0D0E061E08DE00E94652A60E0CA
:103190008DE01C161D06BCF40E94652A64E670E0F2
:1031A00080E090E00E94DA2861E08DE00E94652ACC
:1031B00064E670E080E090E00E94DA2801151105D5
:1031C00031F32197E4CFDF91CF911F910F910C94B0
:1031D000652A0F931F93CF93DF938C01EC01892B0A
:1031E00011F4C1E0D0E060E08CE01C161D06BCF4D8
:1031F0000E94652A64E670E080E090E00E94DA2890
:1032000061E08CE00E94652A64E670E080E090E076
:103210000E94DA280115110531F32197E4CFDF91DF
:10322000CF911F910F910C94652A8091B93590919F
:10323000BA35A091BB35B091BC350196A11DB11D29
:103240008093B9359093BA35A093BB35B093BC3514
:1032500040910401509105016091060170910701B0
:10326000481759076A077B0720F51092B935109265
:10327000BA351092BB351092BC356091BE35809145
:103280000901861780F081E08093BD358091BD35BE
:10329000680F6093BE3570E08CE00E94792960E091
:1032A0008DE00C94652A80910801681778F38FEF00
:1032B000EBCF08958091B9359091BA35A091BB3587
:1032C000B091BC350196A11DB11D8093B935909385
:1032D000BA35A093BB35B093BC35409104015091F1
:1032E00005016091060170910701481759076A07A7
:1032F0007B0720F51092B9351092BA351092BB3584
:103300001092BC356091BE3580910901861780F01E
:1033100081E08093BD358091BD35680F6093BE35E7
:1033200070E08DE00E94792960E08CE00C94652AC1
:1033300080910801681778F38FEFEBCF089560EC68
:1033400070E085EE99E30E94531866E070E085EE28
:1033500099E30E9453186091CD3970E085EE99E3AE
:103360000E94531860EC70E085EE99E30C945318BA
:1033700060EC70E085EE99E30E94531867E070E01E
:1033800085EE99E30E9453186091150170E085EE77
:1033900099E30E94531860EC70E085EE99E30C9479
:1033A000531860EC70E085EE99E30E9453186FE0CB
:1033B00070E085EE99E30E94531861E070E085EEBD
:1033C00099E30E94531860EC70E085EE99E30C9449
:1033D000531860EC70E085EE99E30E9453186FE09B
:1033E00070E085EE99E30E94531870E060E085EE8E
:1033F00099E30E94531860EC70E085EE99E30C9419
:10340000531860EC70E085EE99E30E9453186EE06B
:1034100070E085EE99E30E9453188091CB3961E00A
:1034200070E0811102C070E060E085EE99E30E94D7
:10343000531860EC70E085EE99E30C94531860EC3F
:1034400070E085EE99E30E94531868E070E085EE25
:1034500099E30E94531866E470E085EE99E30E94B8
:10346000531860EC70E085EE99E30C94531860EC0F
:1034700070E085EE99E30E94531860E570E085EEF8
:1034800099E30E94531861E070E085EE99E30E9491
:10349000531862E170E085EE99E30E94531860ECE6
:1034A00070E085EE99E30C9453188091CD39882310
:1034B00041F06091D6397091D7398CE891E00C9445
:1034C000380408958091CD39882341F06091180126
:1034D000709119018CE891E00C9411050895809386
:1034E000C939882321F081E08093CA390895109268
:1034F000CA3908958091CD398823E1F08091C83987
:10350000843A51F4609116017091170150E040E047
:103510008CE891E00E94DF058091C839893A51F426
:10352000609116017091170141E050E08CE891E044
:103530000C94DF0508958091CD39882361F08CE8E3
:1035400091E00E940A026093D2397093D33980933C
:10355000D4399093D53908958091CD39882371F06D
:103560004091D2395091D3396091D4397091D53985
:103570008CE891E00E9477040C949B1A0895809146
:10358000CD39882361F08CE891E00E94DA016093E4
:10359000CE397093CF398093D0399093D139089533
:1035A0008091CD39882371F04091CE395091CF3937
:1035B0006091D0397091D1398CE891E00E94460336
:1035C0000C94BF1A08958091CD39882321F08CE89E
:1035D00091E00C94590280E0089583ED9FE00E94F1
:1035E000511891E0833709F090E0892F0895C8E3DE
:1035F000DFE06FEFCE010E943D182196C11580E1FA
:10360000D807B9F70E9462180E945E18FBCF88E3C2
:103610009FE00E94511891E0833009F090E0892FDB
:10362000089589E39FE00E945118982F8093C8392C
:1036300081E0943A21F0993A11F080E008950895DC
:103640008AE39FE00E9451188093C7399FEF980F3B
:1036500081E09E3F08F080E00895BF92CF92DF9214
:10366000EF92FF920F931F93CF93DF938BE090E045
:103670000E9439277C018C01C8E3DFE0CE010E9463
:103680005118F80181938F012196C334FFE0DF07C1
:10369000A9F76BE070E0C7010E940418B82EC92E8C
:1036A000082F192FDD24D394CE010E945118F80160
:1036B00091918F018913D12C2196C335FFE0DF074B
:1036C00099F78B2D9C2D0E94D527C7010E94D527E5
:1036D0008D2DDF91CF911F910F91FF90EF90DF9093
:1036E000CF90BF9008958FED9FE00E94511891E018
:1036F000833709F090E0892F0895CF92DF92EF92FF
:10370000FF92CF930E94731B882309F461C084ED5C
:103710009FE00E94511890E09093D7398093D6395A
:1037200085ED9FE00E94511890E0909319018093DD
:10373000180186ED9FE00E94511890E090931701C8
:10374000809316018BED9FE00E945118C82F8CEDDD
:103750009FE00E94511890E0B0E0A0E07C01DD24E1
:10376000CC24FC2A8DED9FE00E945118C82F8EEDCD
:103770009FE00E945118C82ADC2AC092CE39D0920C
:10378000CF39E092D039F092D13987ED9FE00E9495
:103790005118C82F88ED9FE00E94511890E0B0E0CA
:1037A000A0E07C01DD24CC24FC2A89ED9FE00E946E
:1037B0005118C82F8AED9FE00E945118C82ADC2AB0
:1037C000C092D239D092D339E092D439F092D5391F
:1037D000CF91FF90EF90DF90CF9008958091CC39FA
:1037E000882309F48AC08091CD39882309F485C0E3
:1037F0006091D63984ED9FE00E943D1860911801D8
:1038000085ED9FE00E943D186091160186ED9FE0D6
:103810000E943D186091D2397091D3398091D4398A
:103820009091D539692F77278827992787ED9FE0D1
:103830000E943D186091D2397091D3398091D4396A
:103840009091D539BC018827992788ED9FE00E9487
:103850003D186091D2397091D3398091D4399091CB
:10386000D539672F782F892F992789ED9FE00E94FE
:103870003D186091D2398AED9FE00E943D18609119
:10388000CE397091CF398091D0399091D139692F4B
:103890007727882799278BED9FE00E943D1860913C
:1038A000CE397091CF398091D0399091D139BC0106
:1038B000882799278CED9FE00E943D186091CE39B2
:1038C0007091CF398091D0399091D139672F782F6D
:1038D000892F99278DED9FE00E943D186091CE3988
:1038E0008EED9FE00E943D1863E78FED9FE00E9400
:1038F0003D188AE090E00C94E9188AE090E00C947E
:10390000B91860E08FED9FE00C943D1882E390E0E1
:103910000E946A180E94F71A8091CA3970E060E02C
:10392000882319F06091C93970E08CE891E00C941B
:1039300085058CE891E00E9442031092CD390895EC
:103940008091CE399091CF39A091D039B091D139B1
:10395000892B8A2B8B2BE1F08091D2399091D3392E
:10396000A091D439B091D539892B8A2B8B2B81F03A
:1039700080911601909117018F3F910549F0809138
:10398000D6399091D739892B19F0109215010895E5
:1039900081E08093150108958091B3018A3F50F42E
:1039A0002091B1013091B20181E02115384118F424
:1039B00080E0089581E00895CF938CE891E00E9423
:1039C0004F01C82F0E94A9286093C4357093C53554
:1039D0008093C6359093C735C0FF2DC081E080939A
:1039E000CF358093CE358093CD358091C835909179
:1039F000C9352091CF35211108C02091CE35211134
:103A000004C02091CD35222319F120910F0130916E
:103A1000100182179307B0F401969093C9358093F3
:103A2000C83581E08093CC358091CB358823E9F08F
:103A3000CF910C945A181092CF351092CE35109227
:103A4000CD35D3CF81E08093CC358093CB35ECCF8F
:103A5000009741F001979093C9358093C835109233
:103A6000CC35E2CF1092CB35FACFCF910C945E18C3
:103A70000F931F930E94A9280091C4351091C5355A
:103A80002091C6353091C735601B710B820B930BAB
:103A900000910B0110910C0120910D0130910E014C
:103AA000601771078207930720F01F910F910C9404
:103AB000DC1C1F910F9108951092900089E1809372
:103AC000910080E89EE3909397008093960080E2B7
:103AD000809371000895809109018093BE35089507
:103AE000803C61F46BED70E085EE99E30E94531821
:103AF0008CED682F85EE99E30C941D2B8B3DC9F757
:103B00006BED70E085EE99E30E9453188DEDF1CFD7
:103B100060EC70E085EE99E30E94531861E270E07A
:103B200085EE99E30E9453188091D7350E94701D4D
:103B30008091D6350E94701D8091D5350E94701DF0
:103B40008091D4350E94701D60EC70E085EE99E3A1
:103B50000C94531860EC70E085EE99E30E945318C2
:103B600062E270E085EE99E30E9453188091D335AC
:103B70000E94701D8091D2350E94701D8091D135B8
:103B80000E94701D8091D0350E94701D60EC70E025
:103B900085EE99E30C945318CF93C0911201C3564C
:103BA00060EC70E085EE99E30E94531863E270E0E8
:103BB00085EE99E30E9453188C2F0E94701D60ECD3
:103BC00070E085EE99E3CF910C94531860EC70E0AF
:103BD00085EE99E30E94531864E270E085EE99E364
:103BE0000E9453188091C6390E94701D60EC70E0ED
:103BF00085EE99E30C94531860EC70E085EE99E340
:103C00000E94531862E070E085EE99E30E94531819
:103C10008091D5390E94701D8091D4390E94701D09
:103C20008091D3390E94701D8091D2390E94701DFD
:103C300060EC70E085EE99E30C94531860EC70E052
:103C400085EE99E30E94531861E070E085EE99E3F8
:103C50000E9453188091D1390E94701D8091D039F3
:103C60000E94701D8091CF390E94701D8091CE39C5
:103C70000E94701D60EC70E085EE99E30C9453187F
:103C8000CF93DF93C8E3DFE0CE010E9451180E947A
:103C9000701D2196C11580E1D807B1F7DF91CF9152
:103CA000089560EC70E085EE99E30E94531861E599
:103CB00070E085EE99E30E9453180E94401E60EC6C
:103CC00070E085EE99E30C945318CF93C82F60EC05
:103CD00070E085EE99E30E94531860E970E085EE8C
:103CE00099E30E9453186C2F85EE99E30E941D2BD7
:103CF00060EC70E085EE99E3CF910C945318CF936C
:103D0000DF93C82FD62F0E94ED1A81110BC0C83C3B
:103D100048F48C2F90E06D2F885C904FDF91CF910D
:103D20000C943D1883E0DF91CF910C94651E0E94A6
:103D3000A01C8091CD3981111DC080911501811188
:103D400038C08091CC398823A1F14091CE3950916F
:103D5000CF396091D0397091D1398CE891E00E94CF
:103D60009503892B41F481E00E94651E90E080E07C
:103D70000E946A18089581E08093CD390E947A1AD2
:103D80000E94AC1A0E94551A0E94621A0E94BF1A21
:103D90008CE891E00E9433056AE272E28CE891E0DF
:103DA0000E94D7020E948C1C83E090E00E94E918D8
:103DB000E1CF83E090E00E94B918DCCF60EC70E0C6
:103DC00085EE99E30E94531864E070E085EE99E374
:103DD0000E9453186091D63985EE99E30E941D2BFD
:103DE00060EC70E085EE99E30C94531860EC70E0A1
:103DF00085EE99E30E94531865E070E085EE99E343
:103E00000E9453186091180185EE99E30E941D2BC2
:103E100060EC70E085EE99E30C94531860EC70E070
:103E200085EE99E30E94531869E070E085EE99E30E
:103E30000E9453186091C93985EE99E30E941D2BA9
:103E400060EC70E085EE99E30C94531860EC70E040
:103E500085EE99E30E94531863E070E085EE99E3E4
:103E60000E9453186091160185EE99E30E941D2B64
:103E700060EC70E085EE99E30C945318CF93C82F53
:103E800060EC70E085EE99E30E94531860E470E006
:103E900085EE99E30E9453186C2F85EE99E30E94FA
:103EA0001D2B60EC70E085EE99E3CF910C945318D4
:103EB0009091C135992309F47BC2803C09F0ACC0D4
:103EC00080910A0181119DC01092C1358091AC1D75
:103ED0009091AD1D6091A81D7091A91D861797073F
:103EE00061F42091AE1D3091AF1D8091AA1D90917B
:103EF000AB1D2817390709F45EC22091AE1D309121
:103F0000AF1D8091AC1D9091AD1D02972817390708
:103F100009F451C28091B1019091B201811598418B
:103F200008F049C22091AD013091AE018091AF01FE
:103F30009091B001019710F48FEF97E182179307EA
:103F400009F44BC02817390708F042C0821B930BB5
:103F50000196009709F42FC24091B3014F5F40933F
:103F6000B301E091AE1DF091AF1D318320834091EC
:103F7000AE1D5091AF1D2091AA1D3091AB1D42176F
:103F8000530771F57093AF1D6093AE1DE091B01BA8
:103F9000F091B11B918380832091B01B3091B11BB4
:103FA0008091AC1B9091AD1B2817390721F58091AA
:103FB000AA1B9091AB1B9093B11B8093B01B809177
:103FC000AF019091B0019093AE018093AD0108953F
:103FD000821B930B8F5F974EBCCF81E090E0BCCFEC
:103FE0002091AE1D3091AF1D2E5F3F4F3093AF1D1E
:103FF0002093AE1DCBCF8091B01B9091B11B029648
:10400000DACF81E08093C1358EEF80930A01109260
:10401000C3351092C23508952091C2353091C33511
:10402000243F91E0390708F0C6C190910A0121159B
:10403000310529F49E3F19F480930A0108959111E6
:1040400046C08B3D21F481E08093C0350895909166
:10405000C035992349F08C3D21F08D3D19F48BED4D
:1040600001C080EC1092C0359091B3019A3F08F0E6
:10407000A2C12091B1013091B2012115384108F05F
:104080009AC12091B1013091B2012F5F3F4F30931F
:10409000B2012093B1012091AF013091B001A9018B
:1040A0004F5F5F4F5093B0014093AF012C543E4F90
:1040B000F90180838091AF019091B0018115984101
:1040C00009F079C11092B0011092AF0108959130BA
:1040D00009F044C08B3DD1F49093C0358091C23536
:1040E0009091C335049709F066C16091CC37709107
:1040F000CD378091CE379091CF370E947A2E6115BF
:10410000710581059105D9F40C941E1E9091C0355E
:10411000992349F08C3D21F08D3D19F48BED01C0C0
:1041200080EC1092C035A9014F5F5F4F5093C335AB
:104130004093C2352453384CF9018083CFCF60932C
:10414000CE397093CF398093D0399093D139809103
:1041500014018131C9F60E94D01AD6CF923009F0ED
:1041600045C08B3DD9F481E08093C0358091C23544
:104170009091C335049709F01EC16091CC377091BE
:10418000CD378091CE379091CF370E947A2E61152E
:10419000710581059105D9F40C94FC1D9091C035F1
:1041A000992349F08C3D21F08D3D19F48BED01C030
:1041B00080EC1092C035A9014F5F5F4F5093C3351B
:1041C0004093C2352453384CF9018083CFCF60939C
:1041D000D2397093D3398093D4399093D539809163
:1041E00014018131C9F60E94AC1AD6CF933099F4EC
:1041F0008F3F11F40C94261F823108F081E190E08A
:10420000909317018093160180911401813191F7E9
:104210000E947A1AEFCF9430D1F48F3F11F40C94AE
:10422000DE1E863088F090E08D30910514F08CE031
:1042300090E09093D7398093D639809114018131E1
:1042400071F70E94551AEBCF86E090E0F2CF9530DF
:10425000D1F48F3F11F40C94F61E853088F090E075
:104260008930910514F088E090E0909319018093D3
:10427000180180911401813171F70E94621AEBCF0D
:1042800085E090E0F2CF993021F40E946F1A0C94EF
:104290000E1F963079F48F3F11F40C949F19811101
:1042A00003C00E94991CF9CF813009F084C00E949C
:1042B000971EF3CF913211F40C94881D923211F4B1
:1042C0000C94AA1D933211F40C94CC1D973021F458
:1042D0000E94A01C0C94B819903319F490E00C942F
:1042E000E918903421F40E94E31A0C943E1F983090
:1042F00029F4833709F05FC00C941F1A9E3059F4DB
:10430000813021F48093CB390C94011A8111FCCFB8
:104310001092CB39F9CF9F3041F40E94CC1C81110F
:1043200002C00C94D1190C94E919993529F4883FED
:1043300009F041C00E94861C913511F40C94511E65
:10434000923551F58B3D79F481E08093C0358091B1
:10435000C2359091C335029771F56091CD37809148
:10436000CC370C947F1E9091C035992349F08C3D39
:1043700021F08D3D19F48BED01C080EC1092C03519
:10438000A9014F5F5F4F5093C3354093C23524530B
:10439000384CF9018083DBCF903511F40C94371A37
:1043A000933511F40C94EE1B943529F40C94811C74
:1043B000803C09F426CE089581E08093AA014FB78E
:1043C000F8942091B5353091B6358091B7359091FC
:1043D000B8354FBF28173907F1F0E091B535F091A6
:1043E000B6358091B3359091B435E817F90761F48B
:1043F0008091B1359091B2359093B6358093B535B3
:1044000080810E94581FDBCFE091B535F091B63521
:10441000CF010196F1CF1092AA010895CF93DF93B7
:10442000EC012197A0F08CE891E00E94BF0120915F
:10443000C4393091C539A9014F5F5F4F5093C539D9
:104440004093C4392053384CF9018083EACFDF917F
:10445000CF9108950F931F93CF93DF93EC01809139
:10446000CB398111B5C08CE891E00E94BF01219742
:104470004091110180FF78C09C0154E0359527954B
:104480005A95E1F72F7033274F3FD9F41092C53971
:104490001092C439209311018CE891E00E946601CA
:1044A00090931301809312018CE891E00E945201D5
:1044B0008093C639CE01DF91CF911F910F910C945B
:1044C0000E224213E3CF8CE891E00E946601209116
:1044D000120130911301820F931F97FD019695955C
:1044E000879590931301809312010091C63910E0D3
:1044F0008CE891E00E945201800F912F911D9595BB
:1045000087958093C639CE010E940E228FEF80934B
:1045100011010E94CC1D0E94E61D60EC70E085EE4A
:1045200099E30E94531870E060E085EE99E30E94E1
:104530005318C0EDD7E32091C4393091C539CE016D
:10454000805D974382179307A0F56991603C39F528
:104550006BED70E085EE99E30E9453186CED85EEEB
:1045600099E30E941D2BE7CF4F3F39F01092C539D8
:104570001092C4398FEF809311018CE891E00E9472
:10458000660190931301809312018CE891E00E94E0
:1045900052018093C639CE010E940E22BACF6B3DE4
:1045A000F1F66BED70E085EE99E30E9453186DED26
:1045B000D6CF60EC70E085EE99E30E94531810921C
:1045C000C5391092C439DF91CF911F910F91089591
:1045D0001092C5391092C4398CE891E00E946601AE
:1045E00090931301809312018CE891E00E94520194
:1045F0008093C639CE010E940E220E94CC1D0E94DB
:10460000E61D60EC70E085EE99E30E94531870E0BF
:1046100060E085EE99E30E945318C0EDD7E3209146
:10462000C4393091C539CE01805D97438217930715
:1046300008F0BFCF6991603C61F46BED70E085EEEE
:1046400099E30E9453186CED85EE99E30E941D2BAF
:10465000E6CF6B3DC9F76BED70E085EE99E30E9404
:1046600053186DEDF1CFCF92DF92EF92FF920F933F
:104670001F93CF93DF93EC018091CD39882309F408
:104680007AC08091CB39811154C00E94621860E0D9
:1046900071E080E090E00E94982C162F107FCF3FB1
:1046A000D10508F0116070E060E08CE891E00E94B4
:1046B0006405612F8CE891E00E94B10098EDC92E4D
:1046C00095E3D92EEE24E394F12CC601885D954341
:1046D0008C179D07F0F4F60161916F018CE891E071
:1046E0000E94B100FFEFEF1AFF0A8FEFE816F10406
:1046F00061F78CE891E00E945C0270E060E08CE879
:1047000091E00E946405612F8CE891E00E94B10065
:10471000D9CF8CE891E00E945C020E946618DF917C
:10472000CF911F910F91FF90EF90DF90CF900C945D
:104730008C1C0E946218CF3FD10519F010F0CFEF0A
:10474000D0E08091CA3970E060E08111BE018CE850
:1047500091E00E94640508ED15E3C801885D95436A
:104760008C179D07B0F6F80161918F018CE891E0FC
:104770000E94B100F2CF82E00E94651E85E090E0C9
:10478000DF91CF911F910F91FF90EF90DF90CF902D
:104790000C946A180F931F93CF93DF938091AB0112
:1047A00081116EC081E08093AB01C0E0D8E14FB7CA
:1047B000F8942091AC1D3091AD1D8091AE1D90916B
:1047C000AF1D4FBF2817390709F45AC0E091AC1D3F
:1047D000F091AD1D8091AA1D9091AB1DE817F907CE
:1047E00009F03FC08091A81D9091A91D9093AD1D27
:1047F0008093AC1D00811181E091AE1BF091AF1B45
:104800002091AC1B3091AD1BE217F30789F5209185
:10481000AA1B3091AB1B3093AF1B2093AE1B2081A2
:104820003181A90141505109443F514008F0BFCFA7
:10483000E8EDF5E3085D1543C8018E0F9F1FBE012B
:104840000E941C2EDC01AC54BE4F8C918193CF0191
:10485000885D95438217930778F3C9010E9433233B
:10486000A6CFE091AC1DF091AD1DCF010296BECF59
:10487000E091AE1BF091AF1B9F012E5F3F4FCBCF5E
:104880001092B3011092B2011092B1011092AB01DB
:10489000DF91CF911F910F9108958091CD39882399
:1048A000E1F10E94381D8091B301882311F18091BC
:1048B000CA35811102C00E94DC1C8091CC35811167
:1048C00028C08091CB35811124C08091CA358823BE
:1048D00031F062E370E080E090E00E94DA280E940C
:1048E000DC1C8091CC35811104C01092CA350E9425
:1048F000CA234FB7F8942091B5353091B6358091E1
:10490000B7359091B8354FBF2817390791F00C94FF
:10491000DC2181E08093CA35ECCF8091CC398823AB
:1049200019F00E941519E5CF0E945A190E94991C8E
:10493000E0CF0895CF938091AC01811127C081E031
:104940008093AC01C4E185EE99E30E94932A892B00
:10495000D9F08FB7F8944091B5355091B635209184
:10496000B1353091B2354217530791F44091B735C4
:104970005091B8352091B3353091B4354217530773
:1049800039F48FBFC150F9F61092AC01CF91089560
:104990004091B7355091B8352091B5353091B63545
:1049A000215031094217530761F38FBF85EE99E318
:1049B0000E94AD2A2FB7F894E091B735F091B83541
:1049C00080834091B7355091B8358091B33590913F
:1049D000B4354817590751F48091B1359091B235EB
:1049E0009093B8358093B7352FBFCCCF8091B73532
:1049F0009091B8350196F4CF1F920F920FB60F9297
:104A000011240BB60F922F933F934F935F936F93A5
:104A10007F938F939F93AF93BF93EF93FF930E94E6
:104A20009A24FF91EF91BF91AF919F918F917F91C8
:104A30006F915F914F913F912F910F900BBE0F900F
:104A40000FBE0F901F901895CF938091863A80FFEC
:104A500029C082E08093BF35C091BF35C130C1F518
:104A60000E94ED1A882381F10E94071B882361F1BF
:104A70000E94111B882341F10E94201B882321F1F1
:104A80000E942D1B882311F1C093CC390E94731B07
:104A90008823E1F00E947D1B82E180931401CF9175
:104AA0000C94971E82FF02C083E0D4CF83FF02C024
:104AB00081E0D0CF42E250E067E371E085EE99E318
:104AC0000E945D2C0E94A4181092CC39CF910895B9
:104AD0001092CC394EE150E06AE571E0EFCF80E012
:104AE0000E945B290E94902CA0EBBDE181E098E13F
:104AF000FD019C01119221503040E1F7E1EBF5E31B
:104B0000B183A083B783A683B583A48380EB95E3A9
:104B10009383828326E040E052EC61E070E085EE12
:104B200099E30E94642B0E945C1D61E08CE00E946E
:104B3000292A61E08DE00E94292AE0EDF7E384EF65
:104B400091E0DF019C011D9221503040E1F7ECEC37
:104B5000F7E384E0DF011D928A95E9F7E4EBF1E0E9
:104B600080E098E1DF019C011D9221503040E1F787
:104B7000A2EBBBE186EF91E0FD019C011192215077
:104B80003040E1F7E8EAFDE1B183A083B783A68373
:104B9000B583A48326EA3DE133832283A4EBB9E104
:104BA000FD019C01119221503040E1F7EAEAFBE15E
:104BB000B183A083B783A683B583A48388EA9BE1EE
:104BC0009383828322E030E043E050E064E070E0D1
:104BD0008CE891E00E94F7000C942425CF93CFB786
:104BE000F8948091DB39811127C0E0EDF0E08491E9
:104BF000E0EBF0E09491E82FF0E0EE0FFF1FEA50B9
:104C0000FF4FA591B491EC91E92321F461E084E098
:104C10000E94652A61E084E00E94292A8CB58061A7
:104C20008CBD8CB580648CBD61E087E00E94292A30
:104C300061E085E00E94292A8091DB398F5F8093B3
:104C4000DB39CFBFCF9108959FB7F8948091DB39BE
:104C5000882319F081508093DB398091DB398111F1
:104C600005C08CB58F7B8CBD1092DA399FBF08953B
:104C70002FB7F894813041F0C0F08230A1F082E08B
:104C80008093DA3980E001C082E09091D939892B94
:104C90008093D9398091DA39811103C081E0809302
:104CA000DA392FBF089584E0F0CF81E0EECF909104
:104CB000DA399230A1F09FB7F894833088F4E82F66
:104CC000F0E0E758FE4F808180952091D93982230A
:104CD0008093D939811102C01092DA399FBF0895AB
:104CE00080E0F2CF0895833060F5E82FF0E0EE0F1A
:104CF000FF1FE65EFE4F71836083813051F082308A
:104D0000A1F0809169008C7F482B40936900E89A5C
:104D1000089580916900837F440F551F440F551FEC
:104D2000482B40936900E99A0895809169008F7C2F
:104D300094E0440F551F9A95E1F7482B4093690082
:104D4000EA9A0895833078F4E82FF0E0813061F03A
:104D5000823061F0E898EE0FFF1FE65EFE4F82E7BB
:104D600096E2918380830895E998F5CFEA98F3CF8E
:104D70001F920F920FB60F9211240BB60F922F9322
:104D80003F934F935F936F937F938F939F93AF93D3
:104D9000BF93EF93FF93E0911A01F0911B010995E6
:104DA000FF91EF91BF91AF919F918F917F916F9103
:104DB0005F914F913F912F910F900BBE0F900FBEBF
:104DC0000F901F9018951F920F920FB60F921124FB
:104DD0000BB60F922F933F934F935F936F937F93F5
:104DE0008F939F93AF93BF93EF93FF93E0911C0139
:104DF000F0911D010995FF91EF91BF91AF919F91A6
:104E00008F917F916F915F914F913F912F910F9073
:104E10000BBE0F900FBE0F901F9018951F920F9210
:104E20000FB60F9211240BB60F922F933F934F930F
:104E30005F936F937F938F939F93AF93BF93EF9302
:104E4000FF93E0911E01F0911F010995FF91EF91F1
:104E5000BF91AF919F918F917F916F915F914F9192
:104E60003F912F910F900BBE0F900FBE0F901F9090
:104E700018950F931F93CF93DF938230910510F411
:104E800082E090E0E091843AF091853A30E020E0D1
:104E9000B0E0A0E0309799F42115310509F44AC03B
:104EA000281B390B24303105D8F58A819B81611587
:104EB000710589F1FB0193838283FE0111C040815A
:104EC00051810281138148175907E0F048175907AB
:104ED00099F4109761F012960C93129713961C9305
:104EE0003296CF01DF91CF911F910F9108950093DA
:104EF000843A1093853AF4CF2115310551F04217C9
:104F0000530738F0A901DB019A01BD01DF01F80167
:104F1000C1CFEF01F9CF9093853A8093843ACDCFFA
:104F2000FE01E20FF31F81939193225031093983DF
:104F30002883D7CF2091823A3091833A232B41F4B2
:104F400020912201309123013093833A2093823AB9
:104F500020912001309121012115310541F42DB717
:104F60003EB74091240150912501241B350BE0915F
:104F7000823AF091833AE217F307A0F42E1B3F0B1D
:104F80002817390778F0AC014E5F5F4F24173507BB
:104F900048F04E0F5F1F5093833A4093823A8193BB
:104FA00091939FCFF0E0E0E09CCFCF93DF93009709
:104FB000E9F0FC01329713821282A091843AB091F9
:104FC000853AED0130E020E01097A1F42081318195
:104FD000820F931F2091823A3091833A2817390724
:104FE00009F061C0F093833AE093823ADF91CF9168
:104FF0000895EA01CE17DF07E8F54A815B819E013B
:1050000041155105B1F7E901FB83EA8349915991B3
:10501000C40FD51FEC17FD0761F4808191810296C2
:10502000840F951FE90199838883828193819B83F3
:105030008A83F0E0E0E012968D919C91139700979F
:10504000B9F52D913C911197CD010296820F931FD6
:105050002091823A3091833A2817390739F63097F0
:1050600051F51092853A1092843AB093833AA09306
:10507000823ABCCFD383C28340815181840F951F74
:10508000C817D90761F44E5F5F4F88819981480F37
:10509000591F518340838A819B8193838283211589
:1050A000310509F0B0CFF093853AE093843A9ECF72
:1050B000FD01DC01C0CF13821282D7CF08951F9269
:1050C0000F920FB60F9211242F933F938F939F93BC
:1050D000AF93BF938091DD399091DE39A091DF3994
:1050E000B091E0393091DC3923E0230F2D3758F5AA
:1050F0000196A11DB11D2093DC398093DD39909379
:10510000DE39A093DF39B093E0398091E139909195
:10511000E239A091E339B091E4390196A11DB11DA6
:105120008093E1399093E239A093E339B093E43965
:10513000BF91AF919F918F913F912F910F900FBE93
:105140000F901F90189526E8230F0296A11DB11D00
:10515000D2CF2FB7F8946091DD397091DE3980910C
:10516000DF399091E0392FBF08953FB7F8948091CF
:10517000E1399091E239A091E339B091E43926B553
:10518000A89B05C02F3F19F00196A11DB11D3FBF7F
:10519000BA2FA92F982F8827BC01CD01620F711D4E
:1051A000811D911D42E0660F771F881F991F4A9548
:1051B000D1F708958F929F92AF92BF92CF92DF92D4
:1051C000EF92FF926B017C010E94B5284B015C01BC
:1051D000C114D104E104F104E9F00E945E280E94A8
:1051E000B528681979098A099B09683E73408105C9
:1051F000910570F321E0C21AD108E108F10888EEA8
:10520000880E83E0981EA11CB11CC114D104E104D6
:10521000F10429F7FF90EF90DF90CF90BF90AF900F
:105220009F908F900895789484B5826084BD84B5F2
:10523000816084BD85B5826085BD85B5816085BD91
:10524000EEE6F0E0808181608083E1E8F0E01082AA
:10525000808182608083808181608083E0E8F0E0EB
:10526000808181608083E1EBF0E0808184608083D5
:10527000E0EBF0E0808181608083E1E9F0E0808113
:1052800082608083808181608083E0E9F0E08081BA
:1052900081608083EAE7F0E08081846080838081A0
:1052A0008260808380818160808380818068808348
:1052B0001092C1000895883020F0873108F487E10A
:1052C00088512091260190E4299F90011124877034
:1052D000822B80937C0080917A00806480937A0096
:1052E00080917A0086FDFCCF8091780090917900C2
:1052F00008951F93CF93DF93182FEB0161E00E9475
:10530000292A209739F460E0812FDF91CF911F91F6
:105310000C94652ACF3FD10511F461E0F5CFE12F60
:10532000F0E0E457FF4FE491E150EA3008F054C058
:10533000F0E0E356F64D0C94712EA729AF29B4295D
:10534000BE29EC29EC29C829D029D829E22984B51D
:10535000806884BDC7BDDF91CF911F91089584B54A
:10536000806284BDC8BDF7CF809180008068809343
:105370008000D0938900C0938800EDCF8091800099
:10538000806280938000D0938B00C0938A00E3CF2B
:105390008091B00080688093B000C093B300DBCFF1
:1053A0008091B00080628093B000C093B400D3CFEE
:1053B00080919000806880939000D0939900C09372
:1053C0009800C9CF80919000806280939000D09324
:1053D0009B00C0939A00BFCFC038D1050CF09DCF81
:1053E00092CF81508A3080F5E82FF0E0E650F64DFC
:1053F0000C94712E0E2A122A042A0A2A242A242AFC
:10540000152A1B2A1F2A252A809180008F778093D6
:1054100080000895809180008F7DF9CF84B58F77CB
:1054200084BD089584B58F7DFBCF8091B0008F77C8
:105430008093B00008958091B0008F7DF9CF809166
:1054400090008F77809390000895809190008F7DD9
:10545000F9CFCF93DF9390E0FC01E455FF4F249107
:1054600084539F4FFC0184918823C9F090E0880FFA
:10547000991FFC01EA50FF4FA591B491FC01E45142
:10548000FF4FC591D49161110DC09FB7F8948C91D5
:10549000209582238C938881282328839FBFDF91C6
:1054A000CF910895623051F49FB7F8943C91822FC8
:1054B000809583238C93E8812E2BEFCF8FB7F894C0
:1054C000EC912E2B2C938FBFEACF1F93CF93DF93BA
:1054D000282F30E0F901E457FF4F8491F901E4559A
:1054E000FF4FD491F901E453FF4FC491CC23A9F0AD
:1054F000162F81110E94F129EC2FF0E0EE0FFF1F13
:10550000E451FF4FA591B4918FB7F894EC9111112C
:1055100008C0D095DE23DC938FBFDF91CF911F9120
:105520000895DE2BF8CFFC01918D228D892F90E01C
:10553000805C9F4F821B91098F7399270895FC010E
:10554000918D828D981731F0828DE80FF11D858D38
:1055500090E008958FEF9FEF0895FC01918D828D6B
:10556000981761F0A28DAE0FBF2FB11D5D968C9183
:10557000928D9F5F9F73928F90E008958FEF9FEFC2
:10558000089586E29CE2892B49F080E090E0892B27
:1055900029F00E94262C81110E94000080E090E0FA
:1055A000892B49F080E090E0892B29F00E940000CF
:1055B00081110C9400000895FC01A48DA80FB92F4F
:1055C000B11DA35ABF4F2C91848D90E001968F732B
:1055D0009927848FA689B7892C93A089B1898C914A
:1055E00080648C93938D848D981306C00288F38910
:1055F000E02D80818F7D80830895CF93DF93EC0130
:10560000888D8823B9F0AA89BB89E889F9898C91AA
:1056100085FD03C0808186FD0DC00FB607FCF7CF66
:105620008C9185FFF2CF808185FFEDCFCE010E9466
:10563000DC2AE9CFDF91CF910895EF92FF920F938B
:105640001F93CF93DF93EC0181E0888F9B8D8C8D2E
:10565000981316C0E889F989808185FF11C0EE8909
:10566000FF896083E889F98980818064808381E093
:1056700090E0DF91CF911F910F91FF90EF900895EF
:10568000F62E0B8D10E00F5F1F4F0F731127E02ECA
:105690008C8D8E110CC00FB607FCFACFE889F98902
:1056A000808185FFF5CFCE010E94DC2AF1CFEB8D02
:1056B000EC0FFD2FF11DE35AFF4FF0820B8FEA89AB
:1056C000FB8980818062D2CFCF92DF92EF92FF92EE
:1056D0001F93CF93DF93EC016A017B01122FE889BE
:1056E000F98982E08083C11481EED806E104F104D7
:1056F000A1F060E079E08DE390E0A70196010E94BF
:10570000302E215031094109510956954795379559
:105710002795211580E1380798F0E889F9891082EA
:1057200060E874E88EE190E0A70196010E94302EB7
:1057300021503109410951095695479537952795CB
:10574000EC85FD853083EE85FF852083188EEC89FE
:10575000FD891083EA89FB89808180618083EA89E1
:10576000FB89808188608083EA89FB8980818068E9
:105770008083EA89FB8980818F7D8083DF91CF914F
:105780001F91FF90EF90DF90CF9008951F920F929E
:105790000FB60F9211240BB60F922F938F939F93F6
:1057A000EF93FF93E091F539F091F6398081E09124
:1057B000FB39F091FC3982FD1DC090818091FE394A
:1057C0008F5F8F732091FF39821741F0E091FE398E
:1057D000F0E0EB51F64C958F8093FE39FF91EF91FD
:1057E0009F918F912F910F900BBE0F900FBE0F9036
:1057F0001F9018958081F2CF1F920F920FB60F92D3
:1058000011240BB60F922F933F934F935F936F9397
:105810007F938F939F93AF93BF93EF93FF9385EE07
:1058200099E30E94DC2AFF91EF91BF91AF919F9184
:105830008F917F916F915F914F913F912F910F9039
:105840000BBE0F900FBE0F901F90189585EE99E339
:105850000E94932A21E0892B09F420E0822F0895E9
:10586000E5EEF9E31382128288EE93E0A0E0B0E067
:1058700084839583A683B78380E891E091838083B6
:1058800085EC90E09587848784EC90E09787868705
:1058900080EC90E0918B808B81EC90E0938B828BFD
:1058A00082EC90E0958B848B86EC90E0978B868BD6
:1058B000118E128E138E148E0895AF92BF92CF92D6
:1058C000DF92EF92FF920F931F93CF93DF936C01C0
:1058D0007B018B01040F151FEB015E01AE18BF08A1
:1058E000C017D10759F06991D601ED91FC91019053
:1058F000F081E02DC6010995892B79F7C501DF916B
:10590000CF911F910F91FF90EF90DF90CF90BF90BC
:10591000AF900895FC01448355836683778308958F
:10592000009729F0BC0190E080E00C94FF2F0895CF
:10593000CF92DF92EF92FF926B017C01C114D104F0
:10594000E104F10441F00E94B02FA70196010E94EA
:10595000522E6B017C01C701B601FF90EF90DF90E2
:10596000CF90089508950E9413290E94B22C0E949E
:105970006F25C1ECDAE20E944D242097E1F30E94EA
:10598000C12AF9CF0E943A2D08F481E008950E94BF
:10599000CE2C6894B1110C94A92D08950E948E2DDF
:1059A00088F09F5798F0B92F9927B751B0F0E1F0E0
:1059B000660F771F881F991F1AF0BA95C9F714C090
:1059C000B13091F00E94A82DB1E008950C94A82D5B
:1059D000672F782F8827B85F39F0B93FCCF38695C9
:1059E00077956795B395D9F73EF490958095709526
:1059F00061957F4F8F4F9F4F0895E89409C097FBA3
:105A00003EF490958095709561957F4F8F4F9F4F95
:105A10009923A9F0F92F96E9BB279395F6958795D9
:105A200077956795B795F111F8CFFAF4BB0F11F49C
:105A300060FF1BC06F5F7F4F8F4F9F4F16C0882343
:105A400011F096E911C0772321F09EE8872F762F79
:105A500005C0662371F096E8862F70E060E02AF0BA
:105A60009A95660F771F881FDAF7880F96958795A6
:105A700097F90895990F0008550FAA0BE0E8FEEF7B
:105A800016161706E807F907C0F012161306E40702
:105A9000F50798F0621B730B840B950B39F40A26FB
:105AA00061F0232B242B252B21F408950A2609F4D9
:105AB000A140A6958FEF811D811D089597F99F67DD
:105AC00080E870E060E008959FEF80EC0895002486
:105AD0000A941616170618060906089500240A9453
:105AE00012161306140605060895092E0394000CD9
:105AF00011F4882352F0BB0F40F4BF2B11F460FF68
:105B000004C06F5F7F4F8F4F9F4F089557FD905890
:105B1000440F551F59F05F3F71F04795880F97FB71
:105B2000991F61F09F3F79F087950895121613062B
:105B30001406551FF2CF4695F1DF08C0161617065A
:105B40001806991FF1CF869571056105089408958F
:105B5000E894BB2766277727CB0197F908950E9421
:105B6000C22D0C94752D0E94672D38F00E946E2D69
:105B700020F0952311F00C945E2D0C94642D1124CB
:105B80000C94A92D0E94862D70F3959FC1F3950F5B
:105B900050E0551F629FF001729FBB27F00DB11DB1
:105BA000639FAA27F00DB11DAA1F649F6627B00D41
:105BB000A11D661F829F2227B00DA11D621F739F2A
:105BC000B00DA11D621F839FA00D611D221F749F38
:105BD0003327A00D611D231F849F600D211D822F7F
:105BE000762F6A2F11249F5750409AF0F1F08823A6
:105BF0004AF0EE0FFF1FBB1F661F771F881F9150D3
:105C00005040A9F79E3F510580F00C945E2D0C94F6
:105C1000A92D5F3FE4F3983ED4F386957795679579
:105C2000B795F795E7959F5FC1F7FE2B880F911DFC
:105C30009695879597F90895AA1BBB1B51E107C05C
:105C4000AA1FBB1FA617B70710F0A61BB70B881F0C
:105C5000991F5A95A9F780959095BC01CD0108959B
:105C6000A1E21A2EAA1BBB1BFD010DC0AA1FBB1F60
:105C7000EE1FFF1FA217B307E407F50720F0A21BD2
:105C8000B30BE40BF50B661F771F881F991F1A943F
:105C900069F760957095809590959B01AC01BD0169
:105CA000CF010895052E97FB1EF400940E94692EE3
:105CB00057FD07D00E94302E07FC03D04EF40C9401
:105CC000692E50954095309521953F4F4F4F5F4F2E
:105CD000089590958095709561957F4F8F4F9F4F58
:105CE0000895EE0FFF1F0024001C0BBE0790F691D5
:105CF000E02D099469279627692778278727782731
:105D000008950E944C2FA59F900DB49F900DA49FC5
:105D1000800D911D11240895E894DF93CF93FC0129
:105D2000DB010E944C2F7F936F93E9019A01AC0134
:105D3000BF93AF933F932F93DF010E944C2F26F424
:105D40006C1B7D0B820B930B9E01EB01FC010E94EF
:105D50005B2FAF91BF912F913F910E945B2FBE01AE
:105D6000CF01F9012F913F91CF91DF910895689470
:105D700001C0E8948F929F92CF93DF930E94C52E2B
:105D8000DF91CF919F908F90089588249924F401FA
:105D9000E401B0E49F93AA279A158B049C04ED05B7
:105DA000FE05CF05D007A10798F4AD2FDC2FCF2F2C
:105DB000FE2FE92D982C892E982F872F762F652F6F
:105DC000542F432F322F2227B85031F7BF9127C0CD
:105DD0001B2EBF91BB27220F331F441F551F661F69
:105DE000771F881F991F881C991CEE1FFF1FCC1F4F
:105DF000DD1FAA1FBB1F8A149B04EC05FD05CE0501
:105E0000DF05A007B10748F08A189B08EC09FD09D7
:105E1000CE09DF09A00BB10B21601A94E1F62EF434
:105E20009401AF01BE01CD01000C0895002E083091
:105E300090F0982F872F762F652F542F432F322FD6
:105E400022270850F4CF220F331F441F551F661F0F
:105E5000771F881F991F0A95B2F7002D089597FDA7
:105E60001094002E083098F00850232F342F452F1F
:105E7000562F672F782F892F912DF4CF1594979552
:105E800087957795679557954795379527950A95FF
:105E9000AAF71124002D0895A29FB001B39FC0015D
:105EA000A39F700D811D1124911DB29F700D811D46
:105EB0001124911D08950E944C2F460F571FC81F93
:105EC000D91F08F4319608958F929F92AF92BF9296
:105ED000CF92DF92EF92FF92CF93DF93EC01688134
:105EE00079818A819B81611571058105910521F474
:105EF00064E279ED8BE597E02DE133EF41E050E08E
:105F00000E94522E49015A019B01AC01A7EAB1E45B
:105F10000E94812E6B017C01ACEEB4EFA5019401CF
:105F20000E943130C60ED71EE81EF91EF7FE06C0CD
:105F300081E0C81AD108E10880E8F80AC882D9824D
:105F4000EA82FB82C701B6019F77DF91CF91FF9074
:105F5000EF90DF90CF90BF90AF909F908F9008957B
:105F60008F929F92AF92BF92CF92DF92EF92FF9269
:105F700060910001709101018091020190910301F3
:105F8000611571058105910521F464E279ED8BE5D8
:105F900097E02DE133EF41E050E00E94522E49019D
:105FA0005A019B01AC01A7EAB1E40E94812E6B016A
:105FB0007C01ACEEB4EFA50194010E943130C60E15
:105FC000D71EE81EF91EF7FE06C081E0C81AD108E8
:105FD000E10880E8F80AC0920001D0920101E09245
:105FE0000201F0920301C701B6019F77FF90EF9085
:105FF000DF90CF90BF90AF909F908F900895609367
:1060000000017093010180930201909303010895B0
:10601000FB01DC0102C001900D9241505040D8F7C5
:106020000895DC0101C06D9341505040E0F70895A0
:10603000F999FECF92BD81BDF89A992780B5089550
:10604000262FF999FECF1FBA92BD81BD20BD0FB694
:10605000F894FA9AF99A0FBE01960895B7FF0C9436
:10606000812E0E94812E821B930B0895F894FFCFFE
:1060700001000000F82A00002801FE030000000FC4
:1060800000FFDCFE1101FF00050072267226722659
:106090000000873A80000100000000B1007602B1E4
:1060A00001BF01B102C7004572726F722C20696E88
:1060B00064657465726D696E61746520626F6F747A
:1060C00020766563746F720D0A004572726F722CD0
:1060D00020696E636F727265637420626F6F7420E3
:1060E000766563746F720D0A0001020400000000FF
:0C60F0001D2B5D2C932AAD2A9F2AFD2A4F
:00000001FF
